:020000040000FA
:100000000000000000000000850107309900031384
:10001000831600308B003F3085007F308100103028
:100020009500FF309000831283169B0183120822F3
:10003000B1000822A8000822A9000822AA00B11FC6
:100040002828B1017430A800E330A9006330AA0069
:10005000640029080F39B2003A226400AD010F3064
:10006000B105AB01310882070E2A0F2A102A122A85
:10007000132A142A162A182A1A2A1B2A1C2A1D2A6D
:100080001E2A1F2AB101B1012D28A42029080F39E9
:10009000AD0203194528AD0082075D285F2861285D
:1000A00063286528672869286B286D286F287128C0
:1000B00073284528452845284528352174283D21A1
:1000C0007428452174284D217428552174285D21F8
:1000D0007428652174286D217428752174287D2168
:1000E0007428852174288D219A212B1895219A2115
:1000F0004528A60CA70CA613AF1CA617F320AF0A21
:100100007928A60CA70CA6132F1DA617F320AF0A5B
:100110008128A60CA70CA6132F1EA617F320AF0A42
:100120008928A60CA70CA613AF1EA617F320AF0AAA
:100130009128A4202908A6002A08A700F320F3206C
:10014000F320F320F32099280C303330C421B30B73
:10015000A6280800C4212908A6002808A700F32023
:10016000AA28B701B70AAB1EB928C4212908033948
:10017000B70735219A21AB1CBE28B8213D219A2111
:1001800045219A214D219A2155219A215D219A21BB
:1001900065219A216D219A2175219A217D219A212B
:1001A00085219A218D219A212B1DD728B8219521AF
:1001B0009A21AB1DEE288D219A2195219A218D211E
:1001C0009A2195219A218D219A2195219A218D217B
:1001D0009A2195219A218D219A2195210000B70B12
:1001E000B928AE21B1283C30A500A61B3521A61F99
:1001F0009521A621261B3D21261F9521A621A61A61
:100200004521A61E9521A621261A4D21261E95219F
:10021000A621A6195521A61D9521A62126195D21E5
:10022000261D9521A621A6186521A61C9521A6218B
:1002300026186D21261C9521A621A71B7521A71F15
:100240009521A621271B7D21271F9521A621A71ACD
:100250008521A71E9521A621271A8D21271E9521CC
:10026000A6219521A50BF528080085018316DB3012
:100270008500831285160511080085018316DD307F
:100280008500831285168510080085018316DE30EF
:100290008500831285160510080085018316F93044
:1002A0008500831205158510080085018316FA3034
:1002B0008500831205150510080085018316FC30A2
:1002C0008500831285140510080085018316DB3034
:1002D0008500831205158512080085018316DD301F
:1002E0008500831285148512080085018316DE308F
:1002F0008500831205148512080085018316F930E4
:100300008500831285140511080085018316FA30D3
:100310008500831205140511080085018316FC3041
:10032000850083120514851008008316FF308500B0
:10033000831208003230A0003208A0076400A10B2D
:100340009E29851DDD29A00B9E2908002830A400C8
:100350006400A40BA829851DDD2908003230A30004
:10036000C42129080F39A3079A21A30BB429080037
:100370000830B5009A21B50BBA2908001030B60034
:100380009A21B60BC02908006400AA0CA90CA80C7D
:10039000281BCD29A818CF29D129A818D129AA17F7
:1003A000D229AA13AA08031D0034A908031D00348A
:1003B000A808031D0034AA170034B10A0F30B10594
:1003C000B00164000000B00BE129851DE1298D21F9
:1003D000EB217D212D28640083169B0183123108B7
:1003E000F9212808F9212908F9212A08F9212122CF
:1003F000080083169A009B0A1C1555309D00AA30F0
:100400009D009C141C1164009C18032A8312080090
:1004100083169B0A1C141A0883120800AA28452870
:100420002B1445289928B128AB14B1282B15B128D5
:10043000AB15B1287928812889289128532AAB1631
:10044000B1288D219A217D219A218D219A217D210A
:100450009A218D219A217D219A218D219A217D2118
:100460009A218D219A217D219A218D219A217D2108
:100470009A2108003521BE213D21BE214521BE2102
:100480004D21BE215521BE215D21BE216521BE2108
:100490006D21BE217521BE217D21BE218521BE2178
:1004A0008D21BE210800A60CA70CA613C421290883
:0A04B00007390319A617F320532A99
:02400E008C3FE5
:00000001FF
